:1000000009C021C034C01FC01EC01DC01CC01BC001
:100010001AC019C011241FBECFE9CDBF10E0A0E661
:10002000B0E0E2E4F3E002C005900D92AE36B10715
:10003000D9F720E0AEE6B0E001C01D92AF36B207BE
:10004000E1F751D07CC1DCCFE82FF0E0E05AFF4F60
:100050008081982F9F7097BB082E000C990B24E08D
:10006000959587952A95E1F78F7088BB08951F9223
:100070000F920FB60F9211240F931F932F933F935C
:100080004F935F936F937F938F939F93AF93BF93A0
:10009000CF93EF93FF93C9E107E010E0D6D0B8010A
:1000A00063D08F5F80936900CFDF8FE295E7019780
:1000B000F1F700C00000C15089F710926E00FF9167
:1000C000EF91CF91BF91AF919F918F917F916F9160
:1000D0005F914F913F912F911F910F910F900FBE04
:1000E0000F901F9018958BB780628BBFAC9A789455
:1000F000BC9885B7877E806185BF81E090E0B4D0F1
:10010000C1E0C80F6C2F81E090E0B5D08C2F90E05B
:10011000A0D010926E0080916E00883240F085B7BA
:10012000806285BF889585B78F7D85BFF2CF80912E
:1001300069008ADF2FE389E191E0215080409040FF
:10014000E1F700C0000080E07FDF2FE389E191E06C
:10015000215080409040E1F700C0000080916E0087
:100160008F5F80936E00D7CF97FB072E16F4009415
:1001700006D077FD08D00BD007FC05D03EF4909553
:1001800081959F4F0895709561957F4F0895AA1BA3
:10019000BB1B51E107C0AA1FBB1FA617B70710F072
:1001A000A61BB70B881F991F5A95A9F780959095A4
:1001B000BC01CD0108958F929F92AF92BF92CF92D2
:1001C000DF92EF92FF92CF93DF93EC016881798108
:1001D0008A819B81611571058105910521F464E295
:1001E00079ED8BE597E02DE133EF41E050E069D008
:1001F00049015A0127EA31E440E050E049D06B015F
:100200007C012CEE34EF4FEF5FEFC501B40140D01D
:10021000DC01CB018C0D9D1DAE1DBF1DB7FF03C0C2
:100220000197A109B04888839983AA83BB839F77EC
:10023000DF91CF91FF90EF90DF90CF90BF90AF9084
:100240009F908F900895B7DF08958AE690E0B3DF1E
:100250000895A0E0B0E080936A0090936B00A093B3
:100260006C00B0936D000895E199FECF8EBBE09ACB
:1002700099278DB30895262FE199FECF1CBA8EBB26
:100280002DBB0FB6F894E29AE19A0FBE019608953D
:10029000EE27FF27AA27BB2708C0A20FB31FE41F22
:1002A000F51F220F331F441F551F9695879577958D
:1002B000679598F37040A9F7009799F7BD01CF01B2
:1002C0000895052E97FB16F400940FD057FD05D026
:1002D00014D007FC02D046F408C0509540953095E4
:1002E00021953F4F4F4F5F4F0895909580957095A2
:1002F00061957F4F8F4F9F4F0895A1E21A2EAA1B41
:10030000BB1BFD010DC0AA1FBB1FEE1FFF1FA217C5
:10031000B307E407F50720F0A21BB30BE40BF50BC2
:10032000661F771F881F991F1A9469F7609570954B
:10033000809590959B01AC01BD01CF010895F89483
:02034000FFCFED
:0E0342000013264C23468C45150701000000D1
:00000001FF
